:100000005A2883169B001C141A08552883169A0038
:100010001C1555309D00AA309D009C149C180E287C
:100020001C115528A301A200FF30A207031CA3073F
:10003000031C55280330A100DF3020201428A10123
:10004000E83EA000A109FC30031C2928A0070318E2
:100050002628A0076400A10F262820182F28A01CFE
:1000600033280000332808000310A10CA00CFF3E29
:100070000318342820085528A20003304528A20080
:1000800001304528A20006304528A8002308210297
:10009000031D4C28220820020430031801300319E4
:1000A00002302805031DFF305528831303138312E4
:1000B0006400080083163F308500303095008113BE
:1000C0008312073099008316FF23900083128B015F
:1000D0000C100B119001D0018316051685168312A2
:1000E000051183160511831205108316051083125E
:1000F0008510831685108312032222216400501A72
:1001000082287C2884207C280515831605118312FB
:10011000DD0164000A305D0203189E285D0801209D
:10012000D3005D083A3E84000008B2006400530822
:10013000320203199C28A328DD0F89280130850687
:1001400083160510831250120130C400C501440803
:10015000A0004508A1000330A300E8303F20031DA4
:10016000B9286400851AB5285016C40A0319C50FAA
:10017000A7286400501EBD28A3280130C400C50173
:100180004408A0004508A1000330A300E8303F2048
:10019000031DD2286400851ACE28A328C40A031997
:1001A000C50FC02805118316051183120800DD0153
:1001B00064000A305D020318E4285D083A3E8400BA
:1001C000FF308000DD0FD828C401C501C40A03191F
:1001D000C50A22216400501AFA284408A0004508E4
:1001E000A100FD30A300E8303C20031DF928E628DB
:1001F000FA2819290511831605118312DD016400FF
:100200000A305D02031811295D083A3E8400000897
:10021000B2005D0883169B00831232080620DD0FB2
:10022000FF280130A300F4301320051583160511B3
:1002300083120330A300E830132005118316051143
:100240008312080050126400851E282908004429E2
:100250000C10CA01CB014A088E004B088F00101405
:100260006400851A3429302910100E08CA000F08BE
:10027000CB004A08A0004B08A1000130A3005E306B
:100280003C20031D442908004A08A0004B08A10097
:100290000430A300E2303C20031D5329E230C600A5
:1002A0000430C70080294A08A0004B08A1000A308A
:1002B000A3008C303C20031D62298430C60003302B
:1002C000C70090294A08A0004B08A1000C30A300E9
:1002D000E4303C20031D7129EE30C6000230C70017
:1002E00090294A08A0004B08A1000C30A300E4307C
:1002F0004220031D8029B030C6000430C700882981
:100300006400851E842980296400851A882984292F
:100310006400851E8C2988296400851A90298C29FF
:10032000DD0164000A305D020318012A0130DE009D
:10033000640005305E020318FF290C10CA01CB01CE
:100340004A088E004B088F0010146400851EB029E7
:10035000640008300F020318AE29A529B029D0295E
:1003600010100E08CA000F08CB004A08A0004B0866
:10037000A1004708A30046084220031DC829D21740
:100380005D083A3E8400520880000310D20CD02948
:10039000D2135D083A3E8400520880000310D20C4C
:1003A0000C10CA01CB014A088E004B088F001014B4
:1003B0006400851ADD29D829FD2910100E08CA000D
:1003C0000F08CB004A08A0004B08A1004708A30073
:1003D00046084220031DF529D2175D083A3E8400E5
:1003E000520880000310D20CFD29D2135D083A3E5A
:1003F0008400520880000310D20CDE0F9829DD0F14
:100400009129501608006400051E072A252A01308C
:10041000CC00CD014C08A0004D08A1001330A30072
:1004200088303F20031D1C2A6400051E182A032A59
:10043000CC0A0319CD0F0A2A05158316051183125C
:10044000D720051183160511831208006300262AA0
:02400E00CC3FA5
:00000001FF
